:1000000077C200000C949D2D90C200008EC20000AB
:100010008CC200008AC2000088C2000086C20000B4
:1000200084C2000082C200000C94D32B0C94BB2C21
:100030000C94882B7AC2000078C2000076C20000BF
:1000400074C2000072C2000070C200006EC20000E4
:100050006CC200000C94AF2B68C2000066C20000A6
:1000600064C2000062C2000060C200005EC2000004
:100070005CC200005AC2000058C2000056C2000014
:1000800054C2000052C2000050C200004EC2000024
:100090004CC200004AC2000048C2000046C2000034
:1000A00044C2000042C2000040C200000501090233
:1000B000A10185020901A1000509190129081500FE
:1000C0002501950875018102050109300931158165
:1000D000257F95027508810609381581257F9501D0
:1000E00075088106050C0A38021581257F95017572
:1000F000088106C0C005010980A101850319012AF4
:10010000B700150126B700950175108100C0050CD8
:100110000901A101850419012AA002150126A002E6
:10012000950175108100C005010906A1018506052C
:100130000719E029E71500250195087501810205D9
:1001400007190029EF1500250195F07501810205B9
:10015000081901290595057501910295017503910D
:1001600001C00660FF0961A1010962150026FF00B8
:100170009520750881020963150026FF00952075FA
:10018000089102C005010906A101050719E029E748
:1001900015002501950875018102950175088101F9
:1001A0000507190029FF150026FF0095067508812F
:1001B000000508190129051500250195057501910E
:1001C00002950175039101C00000000000000000CD
:1001D000000000000000000000000000000000001F
:1001E0000000000000000000000000007E0F00D4AE
:1001F000FFFFFFC7000000780000000000000000C3
:100200002A2B280000000000000000000000000071
:1002100000000029000000002C1E3420212224347C
:100220002627252E362D3738271E1F20212223244E
:1002300025263333362E37381F0405060708090AEA
:100240000B0C0D0E0F101112131415161718191A86
:100250001B1C1D2F3130232D350405060708090A04
:100260000B0C0D0E0F101112131415161718191A66
:100270001B1C1D2F3130354C09025B00030100A00F
:10028000FA09040000010301010009211101000124
:10029000224400070581030800010904010002034C
:1002A000000000092111010001222200070582033C
:1002B00020000107050303200001090402000103D7
:1002C00000000009211101000122B6000705840386
:1002D0002000011201000200000008575002000037
:1002E00001010203011C037600690061006C003A01
:1002F00000660036003400630032006200330063A1
:100300000000000C0353006F0074006B00610000DC
:10031000001C0350006F0068006A006F006C0061F1
:1003200000200057006F0072006B00730000000493
:100330000309040000000000000000000000002984
:10034000001E001F002000210022002B0014001AB4
:1003500000080015001700E000040016000700095F
:10036000000A00E1001D001B000600190005000046
:100370000000000000E30028002C00000000000046
:10038000000000000000002A0027002600250024AD
:100390000023002F00130012000C0018001C003472
:1003A0000033000F000E000D000B00E50038003791
:1003B00000360010001100000000000000E600E51B
:1003C000002800FD377A585A000004E6D6B44602E9
:1003D00000210116000000742FE5A3E0021400ECD8
:1003E0005D003D8889C65436C3174FE4E469645103
:1003F0009AFD9A6CA0E101CD5276615EF74DC5E79A
:100400006A124756AF26249F25862ABB87A3B9ECDC
:10041000DE958B662FB542DF4CA883EBF672175141
:100420008A83CCD486795A1AA22D2E4AA06D816473
:100430002B7EAE133AD52FE027371434CFEF6FFF62
:10044000AFBAE7DA89B2138D92A3971300A7B45F0E
:10045000F0B9021AC3D9FB8BE3FB83FACCA74D0D8D
:100460000736C24A0456383F8E51DFF38E58DDAF4F
:1004700072DD2F537A29B3743BCA03F62CFD570360
:10048000BA964F10806D3F4070BE9A7DFFB409331D
:10049000F2DE5C05454314A7429BC557E1AA5F22E3
:1004A0007BA6C2A4F5249ABA581118F89F7B080BB2
:1004B000330DFDBEC9C86CDCD38896B8567A352793
:1004C000B15BD4BA0E0990B6DF24F6E255E3008E94
:1004D0002C6F89B2DF8CE100018802950400004294
:1004E000A8E1C6B1C467FB020000000004595A002D
:1004F00011241FBECFEFDAE0DEBFCDBF11E0A0E0D8
:10050000B1E0E6E2F0E602C005900D92AC3DB10725
:10051000D9F724E0ACEDB1E001C01D92AB36B207D3
:10052000E1F70E94D7240C949E2F6ACD9C019A95E6
:1005300081159F4118F5F32FF270EE27832F8170FC
:10054000732F74706627532F5870442734FF0CC0E4
:100550008295807FEF2B09F08062672B09F0806421
:10056000452B69F080680895EF2B09F08260672BB6
:1005700009F08460452B19F08860089580E00895A3
:10058000CF93DF93EB01D2DFFE010995DF91CF918D
:100590000895982F92959F7024E0911102C020E059
:1005A000982F892F86958695811511F02E5F982FAB
:1005B000892F8695820F0895809320040895809353
:1005C0002104089521E030E001C0220F8A95EAF766
:1005D00080912104822BF3CF21E030E0A90102C0F9
:1005E000440F551F8A95E2F7CA0180959091210426
:1005F0008923E5CF292F9C3090F5863080F590E057
:1006000036E0239F800D911D1124282F277041E093
:1006100001C0440F2A95EAF723E0969587952A951D
:10062000E1F7FC01EE0FFF1FE80FF91FE152FD4F4C
:1006300020E030E070E05191DF01CB01022E02C0DA
:10064000969587950A94E2F7817081958527842392
:1006500085278E932F5F3F4F2330310561F7089533
:10066000292F9C3078F5863068F590E036E0239F9E
:10067000800D911D1124682F677023E09695879552
:100680002A95E1F7FC01EE0FFF1FE80FF91FE15279
:10069000FD4F40E050E080E0219130E0062E02C0A6
:1006A000369527950A94E2F721703327042E01C06E
:1006B000220F0A94EAF7822B4F5F5F4F43305105B8
:1006C00059F7089580E008959091210421E030E0E9
:1006D000F90101C0EE0F8A95EAF7D90102C0AA0F0D
:1006E000BB1F6A95E2F7EA2B01C0220F4A95EAF791
:1006F000892F8E23E81303C0892F822B60CF20958A
:10070000822F8923FBCF809129049091280498138C
:1007100001C008958F5F8770FACF90912304809570
:10072000892380932304282F2770211110C0891753
:1007300071F090916A0492FF0AC08695869586951D
:100740004BDF109223041092250410922404089584
:1007500090911E04982B90931E040895982F9095C5
:1007600080911E04892380931E04089580911D04A6
:10077000811531F010921D04109227041092260466
:100780000895803E9105D9F1C8F48133910509F4AB
:1007900082C048F48932910509F472C08A32910509
:1007A00009F480C0089589339105E9F082389105F4
:1007B000D1F08533910509F45EC00895843E91051A
:1007C000D9F148F4823E910539F1833E910549F112
:1007D00081EE90E00895863E9105C9F1873E91052E
:1007E00009F43EC00895209169042370211164C06A
:1007F00020916A0423FF14C089E290E008952091BB
:10080000690420FD45C030916A0430FF09C024FD11
:1008100024C083EE90E008952091690422FDF7CF73
:1008200008952091690422FD44C030916A0430FD8E
:1008300043C024FFF5CF11C020916A0421FFF0CFFF
:100840008091690484FD09C087EE90E008952091AD
:10085000690423FFE5CF24FFF7CF80E090E00895FF
:100860002091690423FD2BC030916A0431FFE1CF50
:1008700084EE90E008952091690425FFD1CFBCCF8C
:100880002091690425FD1EC020916A0423FFC8CF72
:1008900089E390E008952091690426FFC1CF8AE2A0
:1008A00090E008952091690426FFBACF81E390E09B
:1008B000089582EE90E0089580EE90E0089586EE2F
:1008C00090E0089585E390E008959091690492FF87
:1008D00010C041E0282F2471243009F040E031E0BD
:1008E000282F2871283009F030E0431711F02CE050
:1008F000822793FF10C041E0282F2471243109F092
:1009000040E031E0282F2871283109F030E043170A
:1009100011F02CE0822730916A0430FF10C051E0C2
:10092000282F2171213009F050E041E0282F287153
:10093000283009F040E0541711F029E0822731FFF8
:1009400010C041E0282F2171213109F040E031E051
:10095000282F2871283109F030E0431711F029E0E1
:10096000822794FD877E08951F93CF93DF9309DF3D
:10097000EC01811522E5920708F052C0811540E58F
:10098000940708F0CDC0803E910520F58D3C91057F
:1009900008F0A1C0883A910570F4853A910508F0F5
:1009A00097C081309105B9F10497813A910598F18A
:1009B000C0E0D0E030C0885A91094B97C8F7C85AB8
:1009C000D0E0CC0FDD1FC059DE4F0990D881C02D7B
:1009D000D46421C0811550E49507B0F4C11580E2BC
:1009E000D80708F0B3C0C83ED105A8F0CE019A954B
:1009F00081159F41E8F68D2F68DF182FCE019927CA
:100A0000C0DEEC01D12B07C09927BBDECC27DF70FD
:100A1000C82BD92BD06ACE01DF91CF911F910895B9
:100A2000803842E59407C8F5803652E5950708F00E
:100A30005BC0C03482E5D807D0F4C03292E5D90754
:100A400008F04BC08C2F8695869520E2829FC001CE
:100A50001124C37021E030E0A90102C0440F551FEA
:100A6000CA95E2F7EA01C82BD92BDD68D4CF8C2FC9
:100A700086958695877050E2859FC0011124C370CA
:100A800021E030E0A90102C0440F551FCA95E2F7EA
:100A9000EA01C82BD92BDC68BECF803C52E5950714
:100AA00058F48F71C03AD245A0F590E0982F88276E
:100AB000EC01C46FD06AAFCF805C9245809708F09C
:100AC00077CFDC2FCC27CC27DF71C06FD06AA3CFC4
:100AD000A497D064A0CFD0659ECFCF71D0E0DC2F9B
:100AE000CC27C16FD06A97CF86958695877020E214
:100AF000829FC0011124C37021E030E0A90102C02F
:100B0000440F551FCA95E2F7EA01C82BD92BDA68C2
:100B100082CFDBDEC82FD0E0DC2FCC27D0627BCFAA
:100B20008F71D3DE93E0CC0FDD1F9A95E1F7CC27D0
:100B3000DF70282F30E084FF05C050E1859F9001D1
:100B400011243327C22BD32BD06965CF8D2F8F7102
:100B5000BCDE182FCE01992714DEEC01D12BDECF9D
:100B600080E00895F894E82FE295EF70F0E041A15D
:100B70008F7021E030E0B90102C0660F771F8A95BF
:100B8000E2F7CB01962F9095942391A392A1892B04
:100B900082A37894089581152CE7920741F420915F
:100BA000710230917202232B11F480E090E00895DD
:100BB000E6E9F3E080E090E065EF73E248E154E2BB
:100BC0002AE834E277836683518740873387228718
:100BD00097878687019670968830910599F70895D2
:100BE000FC018481862381110AC082818115B9F0BC
:100BF0006823908593FF05C081E061110FC080E0FC
:100C00000895282F22952F708F70282B962F92955C
:100C10009F706F70962B81E02913F1CF089581E0CA
:100C200008950F931F93CF9301E010E0082E01C0A9
:100C3000000F0A94EAF7C0911C049C2F9023911195
:100C400015C090912304969596959695891306C0A4
:100C5000109223041092250410922404B3DCC027C0
:100C6000C0931C04CF911F910F910895B5DCF7CF6D
:100C7000282F35EB2303C001112497FF04C08058AF
:100C80009109892F089580589F4FFBCF8091FC02D6
:100C900080FD14C081FD14C082FD16C08091FB024E
:100CA000811581F08E3180F420E5829FC0011124EE
:100CB0006EE170E00E94E32E862F089584E108958E
:100CC00088E2089588E0089580E508958091FC0207
:100CD00080FD17C081FD17C082FD19C08091FA0206
:100CE000811599F0883298F428E0829FC001112480
:100CF00068E270E00E94E32E6115710551F0862FC5
:100D0000089562E0FCCF64E0FACF61E0F8CF68E0DC
:100D1000F6CF81E00895FA01309709F0099508951A
:100D20008091A902811569F0E091D502F091D60277
:100D3000309739F00190F081E02D309711F009954E
:100D4000089580E00895A3E0B0E0E9EAF6E00C94AD
:100D5000BC2E9C0180912C0290912D02821793074A
:100D6000B1F030932D0220932C02E091D502F09146
:100D7000D602309761F00084F185E02D309739F08C
:100D800083E089833B832A83CE01019609952396CC
:100D9000E2E00C94D82EA3E0B0E0E1EDF6E00C9494
:100DA000BC2E9C0180912A0290912B0282179307FE
:100DB000B1F030932B0220932A02E091D502F091FA
:100DC000D602309761F00084F185E02D309739F03C
:100DD00084E089833B832A83CE010196099523967B
:100DE000E2E00C94D82E90914701913091F0A0EE62
:100DF000B1E0EFEF90E02D91821751F0EF3F19F441
:100E0000211101C0E92F9F5F9630A9F7EF3FC9F488
:100E100008959091690497FFEACFE82FE695E6954B
:100E2000E695803FA8F7F0E0EA51FE4F877021E099
:100E300030E001C0220F8A95EAF78281822B8283FB
:100E400008950E2E000CFF0BE252FE4FF8CF90914A
:100E50004701913021F49091690497FD0CC0E0EEB8
:100E6000F1E09191891302C0DF011E9251E0E63E4C
:100E7000F507B9F70895E82FE695E695E695803FE2
:100E8000C8F7F0E0EA51FE4F877021E030E0A90199
:100E900002C0440F551F8A95E2F7CA0180959281DE
:100EA0008923828308958091460108952FB7F8948D
:100EB0008091260290912702A0912802B0912902E8
:100EC0002FBF0895CF93DF93C0911E048091220419
:100ED000C82B80911D048115F1F0E8DF20912604D4
:100EE00030912704821B930B8838934108F03EDC35
:100EF000D0911D0480914701813021F480916904D3
:100F000087FD13C086E020EE31E090E0815088F448
:100F100091112CDCCD2B8091120380958C23909124
:100F20001103892BDF91CF9108958EE128EE31E0F6
:100F3000ECCFF90141919F01411541F39F5FE6CF4D
:100F4000962F20916A0422FF0EC0682F660F660F4D
:100F5000660F692B6093230435DBA8DF909325048B
:100F60008093240408952ECB90911D04292F2823CB
:100F7000211559F08095892380931D04811531F046
:100F800095DF8093260490932704089580E090E0F5
:100F9000F8CF8CDF2091FF0230910003232B211525
:100FA00021F080935E0290935F02209101033091C3
:100FB0000203232B211521F080935C0290935D02A4
:100FC000E091D502F091D602309759F00680F78172
:100FD000E02D309731F082E08093FD028DEF92E0BA
:100FE00009950895611509F441C0E3E3E80FE33181
:100FF00048F4F0E0E056F04D0C94F62E47DE819573
:1010000080930003C6CF42DEFBCF40DE8195809304
:10101000FF02F8CF3BDEFBCF59DE80930103F2CF16
:1010200055DE8195FACF52DE819580930203EACF97
:101030004DDEFBCF815D990B21E030E001C0220F36
:101040008A95EAF78091FE02822B8093FE02DACF26
:101050008091FC0281608093FC02D4CF8091FC02DD
:101060008260F9CF8091FC028460F5CF4091FF024D
:101070008D3C59F48091000387FF0DC0109200034E
:10108000411559F41092FB0208C08E3C81F4809106
:10109000000318169CF3411581F080910103909193
:1010A0000203892B8111AECF1092FA02ABCF8F3C95
:1010B00041F447FFF0CF1092FF02809100038115A9
:1010C000E0CF803D19F41416B4F3E5CF90910103FD
:1010D000893D29F41916FCF610920103DCCF8A3DF4
:1010E00019F497FFD8CFF8CF909102038B3D29F4E4
:1010F00097FFD1CF10920203CECF8C3D19F4191671
:10110000CCF3C9CF9FE2980F983090F4815D990B92
:1011100021E030E0B90102C0660F771F8A95E2F73F
:10112000CB0180959091FE0289238093FE02B3CF7C
:101130008D3D31F48091FC028E7F8093FC02ABCF19
:101140008E3D21F48091FC028D7FF7CF8F3D09F019
:10115000A2CF8091FC028B7FF0CF2FB7F8946091E3
:1011600026027091270280912802909129022FBFB8
:1011700008950F931F938091A902811521F0EDDF4F
:101180001F910F910895E9DF0091AB021091AC021D
:101190002091AD023091AE02600F711F821F931F2C
:1011A000EFCFCF92DF92EF92FF92CF93DF93D82FC2
:1011B000C92FC0909003D0909103E0909203F090DB
:1011C0009303CBDF6C197D098E099F09643F714041
:1011D0008105910510F1C1DF6B017C0182E390E094
:1011E000A0E0B0E0C0925802D0925902E0925A02B8
:1011F000F0925B028093540290935502A0935602A2
:10120000B0935702D0938E03C0938F03DF91CF9199
:10121000FF90EF90DF90CF90089584EF91E0A0E0F1
:10122000B0E0E0CF87E797E790930108809300084C
:1012300088E19AE00FB6F894A895809360000FBEFD
:1012400090936000FFCFFC019B0180911C02909164
:101250001D028617970740F0672B29F48091E8005C
:101260008E778093E800C90140E0009741F4411176
:1012700006C08091E80082FF2FC080E00895209191
:1012800073022115A9F12530A9F12091E80023FD71
:101290002DC02091E80022FDECCF2091E80020FF36
:1012A000E4CF3091F3002091F200009719F028303C
:1012B000310558F041E02830310509F040E0209137
:1012C000E8002E772093E800D0CF41914093F100C1
:1012D00001972F5F3F4FE9CF80917302811541F055
:1012E000853041F08091E80083FFC3CF81E008950D
:1012F00082E0089583E008958091160287FF13C06D
:101300008091E80082FF06C08091E8008B7780938F
:10131000E8000895809173028111F2CF08958091C1
:1013200073028115D9F38091E80080FFF8CF809196
:10133000E8008E77ECCF2091E4003091E50095E64F
:10134000A9012091EC00822F817020FF06C08091BE
:10135000E80080FF06C080E008952091E80022FDAB
:101360001AC080917302811589F0853089F08091CF
:10137000EB0085FD0FC02091E4003091E50042179D
:101380005307F9F29A95E1F684E0089582E0089512
:1013900083E0089581E00895E8EDF0E080818E7F9C
:1013A00080831092E2001092DA001092E100A0EE29
:1013B000B0E08C9181608C9380818F77808319BCA1
:1013C000A7EDB0E08C918E7F8C9380818F7E80839F
:1013D000109215020895E091D502F091D60230974F
:1013E00039F00284F385E02D309711F060E2099521
:1013F0000895FC01AC014A5F5F4F8FEF61E391916B
:10140000892728E030E0982F990F87FF09C0892F9E
:10141000862721503040B9F7E417F50781F7089582
:10142000892FF7CF982F9093E900891771F0709169
:10143000EC002091ED005091F00021FD09C09F5F6C
:10144000973089F78093E9000895762F242F50E094
:101450003091EB003E7F3093EB003091ED003D7F0B
:101460003093ED003091EB0031603093EB007093DE
:10147000EC002093ED005093F0002091EE0027FD4A
:10148000DECF0895A0E0B0E0E8E4FAE00C94B62ED8
:10149000C8EDD0E088818F7E8883E7EDF0E0808121
:1014A0008160808384E082BF81E08093150288811F
:1014B0008E7F888302EE10E0F80110821092DA002D
:1014C00081EEC82ED12CF601108288818F77888317
:1014D00088818068888388818F7D888319BC109279
:1014E000730210921402109246021092130290EEB0
:1014F000E92EF12CF70180818B7F808388818160C8
:10150000888342E060E080E08DDFF60180818E7F9D
:101510008083F801808181608083808188608083FE
:10152000F70180818E7F8083888180618883CDB739
:10153000DEB7E8E00C94D22EE091290490912804C3
:1015400027E0E91302C080E00895AE2FB0E02E9F9F
:10155000F0011124E65DFB4F3181361306C0308166
:10156000381303C03581341304C0FD013196E77090
:10157000E8CF81E008950F931F93CF93DF938B0102
:10158000EA0190917302943051F58093E9008FEF56
:101590009091E80095FD06C095ED9A95F1F7000051
:1015A0008A95B1F78091E80085FF19C0C4DE8111EA
:1015B00011C08091E80085FD06C08091E8008E771B
:1015C0008093E800F3CFF80181918F018093F100BF
:1015D000219779F78091E8008E778093E800DF917A
:1015E000CF911F910F910895792F603229F440E235
:1015F00050E0682F82E0BFCF0895CF93DF93D82FBC
:10160000C92F48E050E0682F792F81E0B4DF88E0EF
:10161000ED2FFC2FAEE1B2E001900D928A95E1F73B
:10162000DF91CF910895BC0140E250E084E0A3CF68
:10163000BC0146E050E084E09ECFBC0143E050E0B6
:1016400084E099CFA0E0B0E0E8E2FBE00C94B42E97
:10165000F82EE92EB62EA72E8A01809110029AE06C
:10166000C92ED12C8A3018F0CC24C394D12CC1E0DF
:10167000D0E06B2D7A2D8F2D9E2DF80109958111CB
:1016800016C02196CC16DD0694F0CC9FC001CD9FEC
:10169000900D900D112420E030E045E34A95F1F7DC
:1016A00000002F5F3F4F28173907B9F7E2CFCDB7BA
:1016B000DEB7EAE00C94D02E90916A0492FB2227C8
:1016C00020F9281771F080FB92F990936A046091D9
:1016D000690470916A0484E090E00E94832F82E0A4
:1016E0001CC808951F93CF93DF93962F122F632F5B
:1016F0008430D8F49C30C8F44630B8F4C42FD0E01D
:10170000CC0FDD1F2CE0929FC00DD11D112490E95C
:10171000899FC00DD11D1124CE0189960E94692F89
:10172000612FCE018A960E94692FDF91CF911F9180
:10173000089580914701813061F58091690487FFA8
:1017400028C0C0DB8093E70140E250E065EB72E027
:1017500086EE91E00E94202F892BD1F080E2E6EE08
:10176000F1E0A5EBB2E001900D928A95E1F7E091EE
:10177000D502F091D602309759F00480F581E02D22
:10178000309731F086E08093E60186EE91E009958E
:10179000089598DB8093DE0148E050E067ED72E049
:1017A0008EED91E00E94202F892B91F388E0EEEDE1
:1017B000F1E0A7EDB2E001900D928A95E1F7E0919A
:1017C000D502F091D602309719F30280F381E02D13
:1017D0003097F1F28EED91E0DACF811519F00E9489
:1017E000A803A7CF0895811531F090912204892B89
:1017F000809322049ECF0895CF93C82F8115C1F006
:101800008CEF8C0F813A80F580914701813021F473
:101810008091690487FD0EC0E0EEF1E08191C81768
:10182000F9F021E0E63EF207C9F78C2FDCDA81DF20
:10183000CF910895EC2FE695E695E695F0E0EA5114
:10184000FE4F828190E04C2F477021E030E002C0D3
:10185000220F331F4A95E2F782239323892B29F322
:101860008C2FF5DA66DFE1CF80E28C0F883048F408
:10187000C77081E001C0880FCA95EAF70E94A803EB
:10188000D6CF8BE58C0F833030F42C2F2452330BC2
:10189000C90159DACDCFE8E5EC0FEB3148F4F0E0BF
:1018A000EE0FFF1FEA55FE4F8081918174DAC0CFA1
:1018B00083E38C0F833108F0BBCF61E08C2F92DB88
:1018C000B7CFCF93DF93EC01805E9109089720F0AA
:1018D00063EF7BE0209711F46DEE7BE0CE010E9478
:1018E000C0028C2F89DFDF91CF910895811541F1DE
:1018F0009CEF980F913A10F4AADA1BCF90E2980F60
:10190000983050F4877091E001C0990F8A95EAF7FA
:10191000892F0E94AE03F1CF9BE5980F933018F406
:1019200080E090E010CA98E5980F9B3118F480E0B1
:1019300090E031CA93E3980F933110F460E052CBFA
:1019400008951F93CF93DF93182FEB0155DF209756
:1019500031F4812FCBDFDF91CF911F9108958FE973
:101960009FE00197F1F700C000002197F0CF8115AB
:1019700019F00E94AE03DDCE0895811539F08095EF
:1019800090912204892380932204D3CE08958091DC
:101990000D03811521F082E2F0DF10920D0308950E
:1019A00010921E0480914701813011F580916904E5
:1019B00087FF1EC0E8EEF1E08EE1DF011D928A95FF
:1019C000E9F780E090E0BFD980E090E0E4D91092A0
:1019D0002204AFDE86E0EDEFF2E0DF011D928A9592
:1019E000E9F71092FB021092FA021092FC02D1CA9F
:1019F000E0EEF1E086E0E1CFD3DF2FEF84E39CE07F
:101A0000215080409040E1F700C0000088E19AE05A
:101A10000FB6F894A895809360000FBE9093600075
:101A2000FFCFAAE2B0E0E7E1FDE00C94BB2E86E137
:101A300092E0FC0101962091F100208322E08E319A
:101A40009207B9F780911702893009F457C0C8F49A
:101A5000823009F4B2C0833009F482C0813081F150
:101A60008091E80083FFE6C08091160290911702F2
:101A70009A3008F0DFC0E92FF0E0ED54F04D0C94FF
:101A8000F62E8A3009F489C08B3051F78091160206
:101A9000813231F780911A0290911B02892B01F754
:101AA0008091E800877F8093E80026DC81E09091B8
:101AB0001802911101C080E08093470171DFD0CFFF
:101AC00080911602813A61F68091E800877F8093C9
:101AD000E80080911A0290911B02892B59F060E076
:101AE00080E090E070E0AFDB8091E8008B7780933E
:101AF000E800B6CF68E08EE192E0F4CF8091160264
:101B0000813209F0ADCF80911A0290911B028D7F36
:101B1000892B09F0A5CF8091E800877F8093E800AA
:101B20008091E80082FF17C09091F3008091F2004D
:101B3000029731F48091F100813011F0863021F468
:101B40008091F100809346018091E8008B7780932B
:101B5000E800D2DB85CF809173028111E1CF80CF85
:101B600080911602813A09F07BCF80911A02909100
:101B70001B02892B09F074CF8091E800877F809346
:101B8000E8008091E80080FFFCCF809147018093BE
:101B9000F1008091E8008E77DACF809116028132D1
:101BA00009F05ECF8091E800877F8093E800A4DB96
:101BB000809119028093450153CF80911602813A9A
:101BC00009F04ECF8091E800877F8093E8008091F4
:101BD000E80080FFFCCF80914501D9CF803889F0A3
:101BE000823841F580911A028F70873018F5809302
:101BF000E9008091EB0085FB882780F91092E900CD
:101C000006C080914602880F90911302892B909113
:101C1000E800977F9093E8008093F1001092F10024
:101C20008091E8008E7723C0811116C08091180240
:101C3000813009F18091E80083FF0AC08091E800BB
:101C4000877F8093E8008091EB0080628093EB00B7
:101C5000AA96E3E00C94D72E823061F780911802A7
:101C6000811581F01092E9008091E800877F8093D0
:101C7000E80042DBDFCF81E0933009F080E0809321
:101C80004602F0CF80911A028F702FEF280F263076
:101C900088F68093E9002091EB0020FFE3CF93309A
:101CA00031F48091EB0080628093EB00DBCF909168
:101CB000EB0090619093EB0021E030E0A90102C0BD
:101CC000440F551F8A95E2F74093EA001092EA000C
:101CD0008091EB008860E8CF8111ACCF10911802A1
:101CE0001F778091E3008078812B8093E3008091BF
:101CF000E800877F8093E800FFDA8091E80080FFAA
:101D0000FCCF8091E30080688093E30083E01111B1
:101D100001C082E0809373028DCF8058823008F03A
:101D200089CF80911802909119028C3D53E095075C
:101D300091F583E08A838AE289834FB7F894DE01C4
:101D4000139620E03EE051E2E32FF0E0509357007D
:101D5000849120FF03C082958F703F5F8F708A301F
:101D6000C0F0895C90E08D939D932F5F243161F7E3
:101D70004FBF8091E800877F8093E8006AE270E0BF
:101D8000CE01019660DA8091E8008B778093E800BD
:101D900051CF805DE7CF292F33272330310509F458
:101DA0004EC078F52130310509F488C08BE590E00C
:101DB000E8E7F2E02230310509F03CCF2091E8005D
:101DC000277F2093E80020911C0230911D0282178A
:101DD000930708F49C0140E02115310509F073C018
:101DE000411171C08091E80082FDCDCF80917302D6
:101DF000811549F2853039F28091E80083FFF2CFF6
:101E0000C2CF80911A0290911B022132310509F450
:101E100046C02232310509F00DCF8330910508F01C
:101E200009CFFC01EE0FFF1FEA5AFE4F0190F0812F
:101E3000E02D8D5A9E4FDC018C9190E010C09C01EA
:101E40003327823021F12330310568F4232BB9F494
:101E5000EFE2F3E0E4918E2F90E0EFE2F3E0009701
:101E600009F4E8CEABCF2330310509F0E3CEE5EE3F
:101E7000F2E0E4918E2F90E0E5EEF2E0F0CFE1E1C8
:101E8000F3E0E4918E2F90E0E1E1F3E0E8CFE3E0CE
:101E9000F3E0E4918E2F90E0E3E0F3E0E0CF8330D5
:101EA000910508F0C7CEFC01EE0FFF1FE45AFE4F6C
:101EB0000190F081E02D89E090E080CF82E190E018
:101EC000E3EDF2E07BCF80917302811509F45BCFE3
:101ED000853009F458CF8091E80083FD54CF80917C
:101EE000E80082FD7FCF8091E80080FF75CF909160
:101EF000F3008091F2002115310519F08830910529
:101F000050F041E0089709F040E08091E8008E77BA
:101F10008093E80061CF44914093F10031962150C5
:101F200031090196E8CF803809F084CE8091E8002D
:101F3000877F8093E800809114028093F10070CE37
:101F4000811178CE10911802123008F073CE809172
:101F5000E800877F8093E80010931402CDD9111513
:101F6000D9F084E08093730242E061EC81E05ADAB8
:101F700042E261EC84E056DA42E261EC82E052DA5D
:101F800042E260EC83E04EDA80917302843051F4D7
:101F900082E0809348014ECE8091E30087FDE1CF3F
:101FA00081E0E0CF81E0F5CFCF93DF93EC014A856C
:101FB0005B856E857F850E948B069B8190958091C5
:101FC00022048923809322048C810E94AE03B1DB1A
:101FD00086E0FE0111928A95E9F7DF91CF9108958D
:101FE000CF93DF93EC018D8181FD13C082608D83DF
:101FF000809122049B81892B809322048C810E94F2
:10200000A80397DB488559856E857F85CE010E94A0
:102010008B0610921704109216048D8180FD02C069
:10202000CE01C2DFDF91CF9108951F93CF93DF934D
:10203000182FA0918C03B0918D03109709F448C01C
:1020400010928F0310928E031092120310921103BC
:102050001696CD91DC911797CE019A9581159F41E7
:1020600008F4D07ED1E0C11101C0D0E01996ED9105
:10207000FC911A97309731F01B966D917C9180E01E
:102080000995D823D11539F08CEF8C0F813A20F5C2
:102090008C2F0E9427071115A1F0E0918C03F0917D
:1020A0008D03808584FD0DC080918B03811549F0DF
:1020B000808191819C01215031092F333E4708F4E2
:1020C00070D837DB10928D0310928C0310928B0323
:1020D000DF91CF911F9108952CDB8C2F07DCDBCF94
:1020E000A2E1B0E0E6E7F0E10C94B12EFE013196FA
:1020F0008CE0DF011D928A95E9F782E6A82E81E047
:10210000B82E8F014F01EE24E394F12C2EE6C22E5F
:1021100021E0D22EF50181915F018F3F09F43EC08D
:10212000F894E82FE295EF70F0E021A18F70A701FD
:1021300002C0440F551F8A95E2F7CA01922F982BCF
:1021400091A392A18095892382A3789400C0E8E6A8
:10215000F1E031E0712C21912F3F79F0A22FA2956F
:10216000AF70A05EB0E08C9190E02F7002C09595AA
:1021700087952A95E2F780FF8DC080E0782A330F9B
:10218000CE16DF0641F7F50182918F3F11F00E94D4
:10219000B20550EA5A95F1F7D8017C920F5F1F4FB4
:1021A000B8E6AB16B1E0BB0609F0B4CF4CE050E0A6
:1021B000B40187E392E00E94202F9C01892B41F01B
:1021C0008CE0F401A7E3B2E001900D928A95E1F76B
:1021D0000091440210E00B591D4F232B09F45CC001
:1021E00081E080930F020E94560790930E02809325
:1021F0000D028091A902811509F4A8C07E01EDE0CD
:10220000EE0EF11C86E0D7011D928A95E9F78091C8
:1022100010028A3008F064C041EF52E1B701C801F2
:1022200011DA811509F480C04DEA52E1B701C80105
:1022300009DA811509F478C04BE753E1B701C80109
:1022400001DA811509F470C04AEC52E1B701C80106
:10225000F9D9811509F468C04DEB53E1B701C80104
:10226000F1D9811509F460C01092100280914302E7
:1022700090E046E050E0B7018B599D4F0E94202F1F
:1022800021E020930C02892B09F041C06296EDE019
:102290000C94CD2E832F72CF80910F02811509F4FB
:1022A000A8CFE0900D02F0900E020E9456078E1902
:1022B0009F09059708F49DCF46E050E067E372E080
:1022C000C8010E94202F892B41F086E0E7E3F2E06D
:1022D000D80101900D928A95E1F710920F0289CFF3
:1022E000C0900A02D0900B020E9456078C199D09DB
:1022F000843F914008F090CF80910C02811531F21B
:1023000086E0F70111928A95E9F710920C02A091EC
:102310004302B0E0AB59BD4F86E0FE013D9601900F
:102320000D928A95E1F7B2CF809110028F3F39F478
:102330000E94560790930B0280930A02DDCF8F5FB5
:10234000809310028A3008F491CFF2CFE0904302DC
:10235000F12CA7014B595D4F7A0186E0F801A3E902
:10236000B2E001900D928A95E1F783E992E041D8BD
:102370008093920286E0E9E9F2E0D70101900D92A4
:102380008A95E1F7C0909F02D090A002E090A10250
:10239000F090A2028091060290910702A09108029B
:1023A000B0910902C816D906EA06FB06B1F0C09240
:1023B0000602D0920702E0920802F09209020E94FF
:1023C000AD08C61AD70AE80AF90AC092AB02D09241
:1023D000AC02E092AD02F092AE028091A302809333
:1023E00021048091A402809320048091A602009190
:1023F000A7021091A8029091A50290931E048093C9
:10240000220480916A0482FF0CC080911D04081789
:1024100041F00E945607909327048093260400936E
:102420001D0480911F04181709F430CF10931F0466
:102430002DCFA0E0B0E0EFE1F2E10C94B62EFA016E
:1024400069017801C82F880FDD0B3097B9F0DE01E4
:1024500093E0AA0FBB1F9A95E1F7A35FBE4F1196B9
:102460008D919C9112978E569D4F2C91422F50E04A
:10247000E217F10508F4AF010E942D2FCE010E9452
:102480003E2E182F8115D9F0E114F104C1F083E03C
:10249000CC0FDD1F8A95E1F7FE01E35FFE4F8381DC
:1024A000482F50E0E816F10408F4A701C35FDE4F9F
:1024B0006C817D816E567D4FC6010E942D2F812F2C
:1024C000CDB7DEB7E8E00C94D22E4F925F926F92B8
:1024D0007F92AF92BF92CF92DF92EF92FF920F93D3
:1024E0001F93CF93DF93F82EEB01A42ED22EE32E71
:1024F000B02EC12E488059806A807B800E94AD0832
:102500006419750986099709643671058105910575
:1025100010F4A11491F000E010E020E030E04B2D29
:102520005C2D6D2D7E2D8F2D84DF811539F00E945D
:10253000AD08688379838A839B8381E0DF91CF91A3
:102540001F910F91FF90EF90DF90CF90BF90AF90D1
:102550007F906F905F904F9008950F931F93CF934C
:10256000DF93D82FC92F46E050E069E972E00E945E
:10257000202F41E0892B09F440E006E010E02D2FE8
:102580003C2F64E872E082E0A0DFDF91CF911F91E1
:102590000F9108950F931F9341E09091A3028091B2
:1025A0002104981301C040E001E010E021E234E092
:1025B0006CE772E084E089DF811581F041E0909161
:1025C000A40280912004981301C040E001E010E0D3
:1025D00020E234E068E772E085E077DF1F910F9139
:1025E00008958F929F92AF92BF92DF92EF92FF92E7
:1025F0000F931F93CF93DF9300D000D000D00F92A2
:10260000CDB7DEB77B0101E010E09E01295F3F4FAF
:1026100040E050E060E070E080E00BDF182F8115B3
:1026200009F443C080908E0290908F02A090900297
:10263000B09091020E94AD08DF80681979098A097B
:102640009B09643671058105910530F483E992E0B8
:102650000E94F9098D1549F106E010E09E012F5FF7
:102660003F4F40E050E060E070E081E0E2DE182F94
:1026700083E992E00E94F9098D1122C0111501F140
:102680000E94AD0860938E0270938F028093900237
:102690009093910286E0FE013196A8E8B2E00190A5
:1026A0000D928A95E1F781E00CC086E0E3E9F2E063
:1026B000DE01119601900D928A95E1F71111EACF92
:1026C00080E096E0E8E8F2E0D70101900D929A955B
:1026D000E1F727960FB6F894DEBF0FBECDBFDF91AE
:1026E000CF911F910F91FF90EF90DF90BF90AF902F
:1026F0009F908F900895A4E0B0E0E1E8F3E10C949E
:10270000B62EC0908002D0908102E0908202F090BC
:1027100083020E94AD086C197D098E099F0911E0A2
:10272000643671058105910518F10E94B908DC0134
:10273000CB010296A11DB11D89839A83AB83BC8313
:1027400000E010E020E030E044E050E0BE016F5FC8
:102750007F4F83E06EDE182F811551F00E94AD0887
:10276000609380027093810280938202909383022F
:10277000812F2496E8E00C94D22EA4E0B0E0E3ECA4
:10278000F3E10C94B62EC0907402D0907502E090E4
:102790007602F09077020E94AD0820911E042983F2
:1027A0006C197D098E099F096436710581059105B3
:1027B00008F041C081E09091A502921301C080E031
:1027C000909122049A83811106C081E02091A60293
:1027D000291301C080E090911D049B83811106C0E4
:1027E00081E02091A702291301C080E090911F048D
:1027F0009C83811104C08091A8028917B9F000E080
:1028000010E020E030E044E050E0BE016F5F7F4F19
:1028100086E00FDE811559F00E94AD0860937402C6
:1028200070937502809376029093770281E02496EC
:10283000E8E00C94D22E81E0C3CF0F931F93CF9387
:10284000DF93843030F56C3020F5463010F5C42F1E
:10285000D0E0CC0FDD1F2CE0629FC00DD11D1124F4
:1028600030E9839FC00DD11D1124CE0189960E94AD
:102870004D2F082F10E0102F0027CE018A960E94BE
:102880004D2F9801282BC901DF91CF911F910F91F6
:10289000089580E090E0F8CF462F672F2091B10295
:1028A0003091B202232B81F4703F39F4403F61F440
:1028B0008091AF029091B00208957C3028F44630A8
:1028C00018F4843008F4B9CF80E090E00895A0E0D7
:1028D000B0E0EDE6F4E10C94B72E7C010091210408
:1028E00080912004082BC3E0D0E010E0C8010C2E3A
:1028F00002C0959587950A94E2F780FD09C021975B
:10290000A8F7D12C8D2DCDB7DEB7E7E00C94D32EF0
:10291000DC2EB7018C2FC0DF0E94B404019779F33D
:10292000F1CF0F931F93CF93FC018581008111811B
:10293000811581F0611571F0C801C9DFC82F682FBA
:10294000C8010E94FA02B8018C2FA6DFCF911F9117
:102950000F910895C8010E943003C82FF4CFCF9380
:10296000DF93D82FC92FB3DF6D2F7C2F95DF0E9407
:10297000B404DF91CF910895FC018481811599F011
:1029800080819181ECDF282F92959F70963099F08D
:1029900060F4925F9F70923030F4203FB1F038F4D1
:1029A00081E0283E38F080E008959A5FF3CF81E01F
:1029B000243FC9F7089591E0213F09F090E081E0BC
:1029C000283E08F080E0892B089581E00895382F93
:1029D000292FCB01A32FB22F873F9105A105B10568
:1029E00020F4875F9C4F0C944D2F80E0089585E282
:1029F00090E00E944D2F883A89F486E290E00E9490
:102A00004D2F8F3A59F487E290E00E944D2F91E0CC
:102A1000873D09F090E0892F8170089580E0FCCF18
:102A2000AAE0B0E0E6E1F5E10C94B22EC0907102AC
:102A3000D090720281E090E09093720280937102D4
:102A400010E083E3A82E83E0B82E00E01AC021E056
:102A500030E0111104C0F401859195919C014F2D36
:102A6000602F812F0E94720BF39482E0880E911CDC
:102A700096E0F912ECCF0F5FECE0AE0EB11C0C301B
:102A800019F04501F12CE3CF1F5F1430D1F61A8203
:102A900019821C821B821E821D8218861F8288EC6E
:102AA00090E09A87898709E612E0CE0101967C01C1
:102AB0004AE050E0B801C7010E94872F065F1F4F10
:102AC0005701093B92E0190799F789E0F701119244
:102AD0008A95E9F78FEF9FEF9E838D8387E08A8742
:102AE0004AE050E0B801C5010E94872F065F1F4FE2
:102AF0000930F3E01F07A1F7D0927202C092710271
:102B00002A96ECE00C94CE2EAAE0B0E0EAE8F5E1DB
:102B10000C94B42E03E113E089EBE82E82E0F82E4A
:102B200097E0B92E2EE2C22E22E0D22EAA24A39440
:102B30004AE050E0B701CE0101960E943D2FF80116
:102B40003896DF018B2D1D928A95E9F789819A814C
:102B5000D80111969C938E938F8112968C93129725
:102B60008D8113968C931397888514968C93149764
:102B7000898515968C9315978B819C8117969C93CC
:102B80008E9316978A8587FD04C01E96DC92CE929E
:102B90001D9780FF02C0F801A08681FF07C0D80101
:102BA00018969C911897926018969C9382FF04C087
:102BB000F80190859460908783FF07C0D80118962C
:102BC0009C911897986018969C9384FF04C0F80114
:102BD00090859061908785FF07C0D80118968C91E9
:102BE0001897806218968C93BAE0EB0EF11C015F87
:102BF0001F4FE9E0EE16E3E0FE0609F099CF2A96B2
:102C0000EAE00C94D02E282FCB01283070F44AE053
:102C1000249F90011124B90167597D4F4AE050E08B
:102C20000E943D2F80E090E008958FEF9FEF089580
:102C3000AAE0B0E0EEE1F6E10C94BC2E9C019755C1
:102C40008115914068F4BE016F5F7F4F822FDBDFFB
:102C5000892B31F489859A852A96E2E00C94D82E46
:102C600088EC90E0F9CFA0E0B0E0E9E3F6E10C9465
:102C7000B72E162FD72FC42FD22E8115A9F040932F
:102C80001A040E9456079093120280931102C77093
:102C900081E001C0880FCA95EAF70E94ED0BCDB71D
:102CA000DEB7E7E00C94D32E90911A04491339C093
:102CB000E0901102F09012020E9456079C012E191A
:102CC0003F097901812F9D2FB3DFE816F90648F5FA
:102CD000D0E2DD0DCD15A1F0C77011E0812F01C04C
:102CE000880FCA95EAF70E94B70CD83048F48D2DAA
:102CF000877001C0110F8A95EAF7812F0E94ED0BB2
:102D000060E070E0802F0E94A10CD83040F62D2D9D
:102D1000277081E001C0880F2A95EAF70E94B70C5E
:102D2000BECFC77081E001C0880FCA95EAF7F6CF21
:102D3000A0E1B0E0EEE9F6E10C94AE2EFE01319692
:102D400080E1DF011D928A95E9F700E110E099E04A
:102D5000A92E93E0B92E27EF422E512C612C712C15
:102D60004F0173016201B1E14B165104610471041A
:102D70001CF080E1C82ED12CA601B501C4010E942F
:102D80005A2FAC0CBD1C0D2C000CEE08FF084C1883
:102D90005D086E087F080150104019F76096E0E169
:102DA0000C94CA2E6FEF85E290E00E94692F6FEFBE
:102DB00086E290E00E94692F6FEF87E290E00E9428
:102DC000692F60E088E290E00E94692F29DEB0DF81
:102DD00068EA85E290E00E94692F6FEA86E290E05F
:102DE0000E94692F67ED87E290E00C94692FA0E0C4
:102DF000B0E0EDEFF6E10C94B52EEC018881811581
:102E000021F1813009F048C08981813059F48A81EB
:102E1000239660E570E0893311F060E070E00E9475
:102E2000A10CECCF823029F48A8123960E94FC0BFE
:102E3000E5CF833029F48A8123960E94760CDECF79
:102E4000843041F022968111D9CFCDB7DEB7E9E0C9
:102E50000C94D12E8A81239620E030E09AE0682FEE
:102E60006053770BAB016A30710560F021153105B5
:102E700051F3EFE9FFE03197F1F700C00000215076
:102E80003109F4CF929FB001939F700D11249A01E4
:102E9000260F371F8991E3CFE82FF0E0E850FE4F6F
:102EA000B490282F26952695269530E0F901E85113
:102EB000FE4FE4908770F12C082E02C0F594E79441
:102EC0000A94E2F7E0FAEE24FF24E0F8F901E85270
:102ED000FE4FC490D12C082E02C0D594C7940A94FA
:102EE000E2F7C0FACC24DD24C0F8F901E853FE4F24
:102EF000049110E002C0159507958A95E2F70170DC
:102F00001127E114F10419F081EE0E94FC0BC114A9
:102F1000D10419F086EE0E94FC0B60E070E08B2D6E
:102F20000E94A10CC114D10419F086EE0E94760C07
:102F3000E114F10419F081EE0E94760C01151105DF
:102F400029F060E070E08CE20E94A10C219656CF3F
:102F5000ACE0B0E0EEEAF7E10C94AD2E7C01DC01D0
:102F600014968C91811509F4BEC161E0C701D9DCCA
:102F70008C01F7018581811521F1809116049091D2
:102F800017040097F1F008171907D9F0FC01FF2783
:102F9000887F9927892B09F072C0A4E0EE0FFF1FEC
:102FA000AA95E1F7EA56FC4F8581846085831183F9
:102FB0000083CF0115D81092220461E0C701B1DC73
:102FC0008C01D70115968C91811509F4E1C0C801D7
:102FD00097578038910508F06BC1003108F072C135
:102FE00066EF70E080E090E0F2DC81116BC1812C33
:102FF000912C5401011146C004E09E012F5F3F4F08
:103000006901D601E02F1D92EA95E9F72401350107
:10301000FFEF4F1A5F0A6F0A7F0AC501B401D7DCC0
:103020008983811509F44EC1813009F0AEC0A50134
:1030300094012E5F3F4F4F4F5F4F2D833E834F8351
:103040005887C301B201C3DC182F8A83811509F4A4
:1030500039C18FEF810F833068F56D817E818F815B
:103060009885B5DC8B83811511F0C601C0DE240183
:10307000350133E0430E511C611C711C49C0E0E076
:10308000F0E092CFB7EF8B169104A104B10409F4DC
:1030900019C1C501B4019BDCEFEF8E1A9E0AAE0A7E
:1030A000BE0A8111EFCF0150A5CF4D805E806F80A9
:1030B00078842EC08BEF810F833098F52401350181
:1030C00043E0440E511C611C711C6D817E818F8117
:1030D00098857DDC8B838115D9F0C301B20177DC43
:1030E0008C83811571F08B819C8181305FEF950716
:1030F00010F0982F8827163071F0173079F00E9461
:10310000EA232401350134E0430E511C611C711C7B
:103110005301420176CF0E949723F3CF0E94B82338
:10312000F0CF143009F0C1CF6D817E818F819885F9
:103130004EDC182F2401350184E0480E511C611C1F
:10314000711CC501B4016D5F7F4F8F4F9F4F3FDCF6
:10315000111509F4B7C0811509F4B4C08150990B59
:103160004FEF489F9001499F300D1124A12FA1508E
:10317000BB0B2A0F3B1F2150310950F2EFE9FFE052
:103180003197F1F700C00000F6CFC60130DEC0CFA6
:10319000011527E5120708F4BAC0011538E5130731
:1031A00008F0F8C7680147E5D41A63E073E08C2D96
:1031B0002ADD892B31F5C601E4E0880F991FEA95D5
:1031C000E1F7FC01EA56FC4F2281213009F05BC097
:1031D0002091030330910403232B99F020910503E0
:1031E00030910603232B69F02091070330910803E7
:1031F0004091090350910A03242B352B232B09F40A
:103200004CC080910D03811509F405C1C0901E04C6
:10321000D0901D040E94560788579C4E90930F0330
:1032200080930E03D70115968C91811509F4F3C094
:103230008D2D8C298D79811121C10115B0E51B07D8
:1032400008F0BBC00115E0E41E0708F01EC1063EF1
:10325000110509F4E0C0C80190528115904208F0B0
:103260001BC1D70116968C91803108F4FFC0C801AC
:103270009927109222048D32910509F0B7C082E09F
:10328000809322040DC1223009F0BBCF20910703A7
:1032900030910803232B09F4B4CFFC01E556FC4F11
:1032A00020812E7F20838A569C4F0E94F00FA9CF49
:1032B00003375CE7150759F580910D038115B9F0C7
:1032C0000E94C70C809123048770811561F0D7019B
:1032D00015968C91811539F080916A0482FF03C0A4
:1032E00082E00E948D032C96E1E10C94C92E10928D
:1032F0001E040E94B6030E94560788579C4E909366
:103300000F0380930E0381E080930D03DBCF023A1D
:1033100082E51807C1F158F4C80190528115904216
:1033200020F1013E110579F1053E110503C0023B74
:10333000B2E51B0709F065CF25EE30E02770332793
:1033400081E090E001C0880F2A95EAF720911003F0
:1033500030910D033115F9F0D70115963C913115D7
:10336000A9F0282B20931003ADCFF701868180317F
:1033700008F047CF812F99278F71992782309105C7
:1033800011F04297D7CF21EE30E0D8CF809582233D
:103390008093100397CF322F3823311509F431CFA2
:1033A000982F90959223909310030E94AE03F701FB
:1033B0008581811509F486CF24CF003EB2E51B0735
:1033C00008F047C0003CE2E51E0728F5003AF2E5A8
:1033D0001F07E8F4003622E51207E8F4C801925509
:1033E00080349105C0F010922204C8018E329105FC
:1033F00008F063C08832910508F050C08E31910505
:1034000008F04EC004974A9708F439CF37C0043B00
:1034100032E5130741F7F7013580311409F457C03D
:103420000E35FCE71F0709F44EC00F352CE71207D5
:1034300051F00D353CE7130709F049C0809149016F
:10344000811509F440C01092490180E00E941510D6
:1034500039CF09374CE7140728F407375CE715071D
:10346000D0F6C1CF0B378CE71807D4CF812F8F71DF
:10347000843189F2863111F4109222040E94C70C23
:10348000809110030E94A803C6CFD70116968C9195
:10349000803108F0ECCEBFCFC801EBCE8A9771F730
:1034A00080911003811531F08091220492E08927E8
:1034B000809322040E94990BAECF8C34910581F346
:1034C0008D329240ECCF81E080934901FBCE809118
:1034D0004901811169C0C80197558115914008F0D3
:1034E000FFC05801F8EFAF22BB24A114B10409F0CA
:1034F000E9CEF801FF2754E0EE0FFF1F5A95E1F7E0
:103500009F012A563C4F6901D70115968C91E556CB
:10351000FC4F908180FB90F99083811509F4D9C10B
:103520000E9456079093190480931804F601828133
:103530008F5F82838091220490911E04892B838364
:1035400080911D0484834681578166857785C601F5
:103550000E948B06D60115968C9181FF5801B0927E
:103560001704A0921604D70115969C91911509F4A1
:103570002AC610921A04980130572332310508F0F8
:103580000DC684E090E00E94552F90936A048093CA
:103590006904F801E150F047E232F10508F0E1C1B9
:1035A000E354F04D0C94F62E380150EE651A710874
:1035B00050901F0480911E04582A80911D04582A9F
:1035C00088E06816710408F05EC098012770332700
:1035D00081E090E001C0880F2A95EAF7311409F4E0
:1035E0004FC0582AD7018D919C910E94300321E051
:1035F00030E0F90102C0EE0FFF1F8A95E2F7FC8769
:10360000EB8720918C0330918D033E832D83409175
:103610009403509195035A87498763E1C62E63E06E
:10362000D62EA12CB12C511005C0D60112968C912A
:1036300081111BC0F601838190E02B853C8582239C
:103640009323892B91F08085982F9770911101C059
:1036500087E038E06316710408F066C0311409F49D
:103660005FC086958170811164C09FEFA91AB90A65
:10367000AFE0CA0ED11CB8E0AB16B104A1F61CC075
:1036800080955822AFCF311038C08091940390912B
:1036900095030817190781F410929503109294036B
:1036A0001092900310929103109292031092930340
:1036B00010928F0310928E0380918C0390918D0352
:1036C000009709F408CFE8E06E16710408F0EBC02B
:1036D000652D0E94F005811103C081E00E94151044
:1036E000F7018581F801E851FC47E730F10508F062
:1036F0003ACFE152F04D0C94F62E109395030093BF
:1037000094030E94AD08609390037093910380939B
:1037100092039093930310928F0310928E0362CFC3
:1037200082FB882780F99FCF311409F49ECF80FF58
:103730009CCFD6018D909C900815190519F4311471
:1037400009F493CFED81FE81EC15FD0509F48DCFD1
:10375000D6011D96ED91FC91309721F08081811565
:1037600009F483CF652DC6010E94F005811509F487
:103770007CCF81E00815190509F080E0482E432030
:103780008114910441F0411006C0E985FA858E1636
:103790009F0609F06ACF80E00E941510D0928D0339
:1037A000C0928C0381E080938B038FE08A9DF001AF
:1037B0008B9DF00D1124ED5EFC4F858180931203EB
:1037C00041100EC08114910459F0808191819C01B7
:1037D00024503109213A310508F049C00E942707D9
:1037E0008FE08A9DF0018B9DF00D1124ED5EFC4F62
:1037F000C680D780C6019A9581159F4110F420EEAE
:10380000D22299249394C60101978F339E4708F0E2
:10381000912C8FE08A9DD0018B9DB00D1124AD5E5F
:10382000BC4F1996ED91FC911A97309731F01B9689
:103830006D917C9181E0099598229114A9F08FE017
:103840008A9DF0018B9DF00D1124ED5EFC4F868169
:1038500097810E94960280931103C60148E0641686
:10386000710440F40E94D1080E94990B0AC00E9482
:10387000760CB6CF0497813A910548F48C2D0E94BE
:10388000F306411409F427CE0E94990B1BCD0E9428
:10389000990B8FE39CE90197F1F700C000008C2D94
:1038A0000E94FC0BEECFDC012D913C910217130717
:1038B00041F4311009C010928B0380E00E94151072
:1038C0000ACE311409F407CEFC01808585FD03CEB4
:1038D000F4CFF9014485558566857785C9010E9435
:1038E0008B06D60115968C9181FF3DCEC6010E94B4
:1038F000D40F80911604909117040817190709F046
:1039000032CE10921704109216042DCE06E221EE4C
:1039100041EE6AE17CE7A7D9D5CC07E225EE45EE7A
:103920006BE17CE7F8CF06E221EE40EE68E17CE750
:10393000F2CF07E225EE44EE69E17CE7ECCF06E248
:1039400021EE42EE6CE17CE7E6CF07E225EE46EEA3
:103950006DE17CE7E0CF08E221E045EE6EE17CE737
:10396000DACF809169048160809369046091690471
:1039700070916A0484E090E00E94832F0E94D00C32
:10398000A1CC80916A04886080936A04EFCF809113
:1039900069048260E9CF809169048460E5CF8091F9
:1039A00069048860E1CF80916A048160EDCF8091E5
:1039B0006A048260E9CF809169048061D5CF8091EB
:1039C00069048062D1CF809169048064CDCF0E9468
:1039D000D00C809169048068C7CF809169048C60A5
:1039E000C3CF80916A048360CFCF809169048E7FBA
:1039F000BBCF80916A04877FC7CF809169048D7F98
:103A0000B3CF809169048B7FAFCF80916904877FAA
:103A1000ABCF80916A048E7FB7CF80916A048D7F8F
:103A2000B3CF809169048F7E9FCF809169048F7D91
:103A30009BCF809169048F7B97CF0E94D00C80919F
:103A400069048F7791CF80916904837F8DCF8091B6
:103A50006A048C7F99CF80916904992782FF93959E
:103A600090FB82F990FB83F97FCF80916A04982FB5
:103A7000909590FB80F990FB81F986CF9091690435
:103A8000892F8F7B96FF80646FCF0E94D00C90911E
:103A90006904892F97FB87F9805866CF61E08EE033
:103AA00090E00E94692F62CF60E0F9CF90916904A5
:103AB000892F8F7E94FF806157CF90916904892F61
:103AC0008E7F90FF816050CF90916A04892F877F0D
:103AD00093FF886059CF89E273C389E27FC30737B8
:103AE000BCE71B07F9F00837ECE71E0731F1980136
:103AF000205E32452032310528F5911123C00F7127
:103B000081E090E09C0102C0220F331F0A95E2F78A
:103B10008901622F83E090E00E94692F802F0E942C
:103B2000DC02D0CB81E0911551F00E94E20243E02B
:103B300062E081E00E946403C5CB82E0F4CF0E9482
:103B4000EC02F5CF40911C0480912104282F30E035
:103B50002095309570E024233723232B19F0482338
:103B600040931C040B373CE7130741F4911509F40B
:103B7000A9CB0E94C9020E941106A4CB003442E5E1
:103B8000140708F055C0003252E5150708F057C079
:103B9000011580E5180750F50115A0E41A0708F093
:103BA00064C0911509F479C00A35FCE71F0709F4D0
:103BB000DDC008F0C2C001303CE7130709F4D4C0EF
:103BC00003304CE7140709F4C9C001151C4709F07C
:103BD00064C00E94D00CAFEFB4E3ECE0A150B04061
:103BE000E040E1F700C000000E9412099801305542
:103BF00021153240B0F6980145E0369527954A9553
:103C0000E1F7822F8F7020911C0430E041E050E0FA
:103C1000082E02C0440F551F0A94E2F724233523CF
:103C2000232B09F4BECF9111A6CF10921E042CCEE7
:103C30009801205C32452032310508F0B2CF802F48
:103C40008F7120911C0430E041E050E0082E02C04A
:103C5000440F551F0A94E2F724233523232B09F43C
:103C6000A0CF911509F42ECB86CFF7018681803144
:103C700008F097CF911111C0212F2F7081E090E0B3
:103C800002C0880F991F2A95E2F720911C0430E0AA
:103C900082239323892B09F015CBF7018581C080FE
:103CA000D180811509F466C0C6010E946714182FDF
:103CB000682FC6010E94FA02B601812F0E944C149F
:103CC0000E94B4048C01D7011596BC9015971696E6
:103CD000AC90A2942FE0A2228091230487708115DA
:103CE00001F1CB2CB114F1F0812F807F803461F091
:103CF00080E2800F8830A8F0812F807E803221F40E
:103D0000023078F0A11469F080916A0482FF09C042
:103D100082E00E948D03809123048770CC24C39499
:103D20008111C12CE12FE295EF70103C08F082C0A8
:103D3000F0E0EA51F04D0C94F62E0B358CE71807A5
:103D4000B9F080916A04002482FF0394802D0C3521
:103D50001C4709F0A2CF0E945C0B9FCF6FEF7FEF53
:103D600080E090E00E94832F0E94FC0C81E0F3CF62
:103D700080E0F1CFC6010E943003182F9DCFB12FF4
:103D8000BF70DB2E103118F0D29490EFD922B1140D
:103D9000A9F0D11459F080E2800F883010F00111A1
:103DA00007C08D2D0E94A8030E94990B802F40C050
:103DB000809122048D2980932204F6CF802F0E94C7
:103DC000760CD114B9F180E2800F883010F0011127
:103DD00004C08D2D0E94AE0306C0D09480912204B1
:103DE0008D21809322040E94990B24C0E12FEF7053
:103DF000DE2E107F103219F0D29480EFD8220115F8
:103E000049F0013009F482C0B11409F48EC0A11444
:103E1000A1F1CCCF80916A0482FD2BC0B11419F1BD
:103E2000D11429F08D2D0E94A8030E94990B80E0E7
:103E30000E94FC0BC11409F4D8C08091230480FDBA
:103E4000D4C0D70115961C928695869586950E94BA
:103E5000E202C7017DD880912304869586958695D8
:103E60000E94EC02C2C080E00E94760CD11411F3D3
:103E7000B0CFB11469F1A11004C08D2D0E94ED0BDB
:103E8000D9CFF1E0AF1210C010911D048D2D812308
:103E9000D81681F20E945607909327048093260437
:103EA0001D2910931D04C6CF25E0A212C3CF8D2D6E
:103EB0000E94ED0B8D2D0E94B40780911F049D2D53
:103EC0009823D91609F4B6CF8D2980931F04B2CF59
:103ED000A11012C08D2D0E94B70C8D2D0E94B40729
:103EE00080911F049D2D9823911509F4A3CFD094A0
:103EF000D822D0921F049ECF31E0A3129BCF809195
:103F00001E048D21811509F495CFE4CFB11429F059
:103F100046E0A41608F08ECFB0CF55E0A51608F005
:103F200089CF8D2D0E94B70C85CFA114D1F3093311
:103F300049F48FEF97EEA3E081509040A040E1F765
:103F400000C00000802F0E94760C74CF812F8695D0
:103F500086958370811561F0813009F06BCFC801BF
:103F60009370B11002C080E090E00E94CB0662CF57
:103F7000C8019370B11002C080E090E00E94A306D7
:103F800059CF6B2D802F0E94F20754CF812F837061
:103F9000811138C0B11027C0402F42954695477017
:103FA000440F440F802F8F70042E01C0880F0A9495
:103FB000EAF7202F207104FF07C02FE030E001C096
:103FC000220F4A95EAF72095169516951370123030
:103FD000A1F0133081F030912004113059F0822B80
:103FE00083230E94DC020E94900660E0C7010E94C9
:103FF000911479C9832B822BF4CF822B90912004CA
:104000008927EFCFB11451F110FFEDCF402F42952A
:1040100046954770440F440F802F8F70042E01C0C7
:10402000880F0A94EAF7202F207104FF07C02FE0C1
:1040300030E001C0220F4A95EAF7209516951695B3
:104040001370123089F0133069F03091210411306F
:1040500041F0822B83230E94DF02C5CF823018F209
:10406000D5CF832B822BF7CF822B909121048927E8
:10407000F2CF1F70B11439F0812F0E94E202802F1D
:104080000E94ED0BB0CF802F0E94B70C812F0E94B1
:10409000EC02A9CF023F71F170F4003FC9F0013F7B
:1040A00091F0B11409F465C0A11409F45FC0802F28
:1040B0000E94FC0B98CF033F21F1043F91F78091C0
:1040C0006A0482FD2AC0812F8F71B11401F316C0DA
:1040D000B11469F0B5E0AB1608F085CF1F7181E02F
:1040E00090E0012E01C0880F0A94EAF7BECFE6E007
:1040F000AE16F2CF812F8F71B110C9CF0E94E202AC
:1041000072CF80E0B11409F4A6CF1F7181E0012EB7
:1041100001C0880F0A94EAF79ECFB114C1F08091D4
:1041200023048770843049F41092230410922504EC
:1041300010922404812F8F71AACFF5E063E0AF16AF
:1041400008F051CF812F8F710E94A0074CCF25E03E
:10415000A21640F010922304109225041092240419
:1041600064E0F0CF81E00E948D033DCF812F8F71FD
:10417000C5CFA114F9F2093349F43FEF47EE53E0FC
:10418000315040405040E1F700C00000802F0E94B5
:10419000760C29CF0337BCE71B070CC90631ECE7C7
:1041A0001E0709F09CCC80911E048A7A91E081114F
:1041B00001C090E090931B04811509F48CCC85E339
:1041C0000E94F30661CB0631FCE71F0709F087CC9C
:1041D00080911B04811509F480CC85E30E94270798
:1041E00053CBA0E0B0E0E7EFF0E20C94B72E809163
:1041F0006804803108F049C080916704811509F492
:1042000044C0C091290487E0D82E809128048C17DF
:10421000E1F1EC2EF12CDC9EE0011124FE01E65DC3
:10422000FB4F84818115B1F19181809163049813D2
:1042300031C090818091620498132CC085818111D6
:1042400029C0028113818091640490916504081B48
:10425000190B60E082E694E00E9491140E94181607
:1042600008171907B8F4809168048F7080618093F3
:104270006804C05DDB4F88818F708061888382E62F
:1042800094E00E94A8170E948303CDB7DEB7E7E051
:104290000C94D32EE7012196C770B7CFADE0B0E004
:1042A000E4E5F1E20C94AF2E8C0186E0F801DE012A
:1042B000189601900D928A95E1F7F801F580E48057
:1042C00082E6882E84E0982E80916604811117C0C2
:1042D000E11491F0F11409F455C1C8010E94BC1415
:1042E000811509F44FC187E0F801A2E6B4E001901E
:1042F0000D928A95E1F775DFFF24F39461C0A280E7
:10430000B380D09067048091640490916504350176
:10431000681A790AD11409F4F0C0C080518060E0B5
:1043200082E694E00E9491140E941816681679069D
:1043300008F09EC0E11401F380916304F8019181BB
:10434000E0906804F0E1EF1608F05BC0981317C026
:1043500090916204F8018081981311C0F1104BC054
:104360008E2D8F7080618093680482E694E00E94B5
:10437000A81780916804F8018683F12C21C0F11000
:104380003AC040E0652D8C2D0E949C0A40E0652DCE
:104390008C2D0E949C0AF82E8111EFCF888599857B
:1043A0000E94AF14292F22952F70903470F49F70C3
:1043B0002230A0F09115B1F0F8019681903190F47F
:1043C0008F2D2D96EFE00C94CB2E2A5F2F7022308C
:1043D00068F0C8010E94A817FD2CF2CF911511F0CA
:1043E000811571F3805E883058F3F3CF803F40F33E
:1043F000815F8330F9CF8091680481608093680485
:10440000BCCF981315C090916204F8018081981375
:104410000FC0F1100DC0E682C8010E94A81787E006
:10442000F801A2E6B4E001900D928A95E1F764CF1D
:10443000C8010E94BC14811509F4A4C0F11409F448
:10444000A1C080916804803208F44DCF809162044D
:10445000909163049A838983BC82AB8280916604C5
:104460008D831E82EF82CE0101960E94A8173BCF5A
:10447000D0906804F0E1DF1650F482E694E00E94E8
:10448000A81787E0F40111928A95E9F776CFE11435
:1044900009F432CF90916304F8018181981311C01F
:1044A00090916204808198130CC0F1100AC0D682EA
:1044B000C8010E94A81787E0F40111928A95E9F7D4
:1044C0001BCFC8010E94BC14811509F45BC0F11414
:1044D00009F458C080916804803208F404CF8091B8
:1044E0006204909163049A838983BC82AB82809139
:1044F00066048D831E82DF82B6CF60E082E694E0A0
:104500000E9491140E9418166816790608F0B9CF17
:10451000E11409F4F1CEF114A9F190916304F801CA
:104520008181981325C0909162048081981320C0E6
:104530008091640490916504A81AB90AF8ECAF164A
:10454000B10408F06CCF8091680480FD68CF8031A1
:1045500008F465CFF8018683982F907F903F09F487
:104560005BCF982F907F905F8F70892B868354CF7D
:10457000C8010E94BC148111B6CE8091680481608C
:1045800080936804C8010E94A817B6CEABE1B0E0E2
:10459000ECECF2E20C94BA2E4E8B5F8B688F798F25
:1045A0008A8F192F9B8F9111109222041D8A86E009
:1045B000FE017696DE011F9601900D928A95E1F735
:1045C0000A8D80916A0482FF1FC00E9456072091C5
:1045D000240430912504821B930B8838934138F0D2
:1045E0008091230482FD03C082E00E948D030E941B
:1045F00056072091260430912704821B930B88389C
:10460000934110F00E94B603011561F00B8B1C8BD7
:1046100061E0CE010F960E94911461E0CE010F96E9
:104620000E9491140B8B1C8B87E0FE013F96DE01EC
:10463000189601900D928A95E1F7CE0108962EDE2C
:10464000811110C0209128043091290487E0FE01D7
:104650003896DE01119601900D928A95E1F78C85CE
:1046600081110BC017E080912904909128048913CF
:104670002BC06B96E4E00C94D62E822F90E001962E
:10468000877099273817190671F40E94D00C109280
:1046900028041092290487E0E2E6F4E0DF011D928D
:1046A0008A95E9F7DFCF97E0929FD0011124A65DAC
:1046B000BB4FFE01319601900D929A95E1F78093E0
:1046C00028040E948303CECF189FC0011124865D69
:1046D0009B4FE4DD811569F28091290490E00196F9
:1046E0008770992780932904BECFA6E0B0E0EBE75E
:1046F000F3E20C94BA2E0E9456078C018091B3020B
:104700009091B4028017910771F019821A820E9469
:104710005607BC0149815A8180E090E037DF109351
:10472000B4020093B3022696E4E00C94D62EA6E0E1
:10473000B0E0EDE9F3E20C94BC2E9093B0028093CC
:10474000AF02811520E2920730F40E94610C269698
:10475000E2E00C94D82E80EF89838A830E9456076A
:104760008160BC0149815A8181E091E00FDFEFCF88
:10477000A6E0B0E0EEEBF3E20C94BA2E8C0190933D
:10478000B0028093AF02011580E21807B0F4802FC9
:104790000E94760CC801805E9109089728F06DEBA5
:1047A0007CE00115110511F467EB7CE0C8010E9463
:1047B000C0022696E4E00C94D62E80EF89838A838B
:1047C0000E9456078160BC0149815A8181E090E0D6
:1047D000DDDEEFCFCF93DF93D82FC92FA8DF8D2F4A
:1047E0009C2FC6DFDF91CF9108950F931F93CF9336
:1047F000DF938C01862F63E073E00E940316892B00
:1048000091F4C0910303D0910403209761F0F80163
:104810008281833039F4CE01DDDFCE01DBDFCE01D2
:10482000D9DF01C0E0F7DF91CF911F910F9108957B
:104830000F931F93CF93DF938C01EB0163E073E041
:104840008C2F0E940316892B09F057C0FE01FF2709
:10485000D80112968C911297E15DFD4F8130A9F439
:1048600015968C9182FD4EC080FF4CC082E0808303
:1048700080910503909106030097B9F4809103039A
:10488000909104030097C9F110C08230A1F51596EC
:104890008C9182FD26C080FD0AC083E080838091D8
:1048A0000703909108030097F1F041DF26C084E0F0
:1048B00080838091090390910A030097B1F780915A
:1048C000030390910403009701F184DF80910503B5
:1048D00090910603009749F7809103039091040398
:1048E000E4CF85E0808380910303909104030097D7
:1048F00021F070DFF1CF86E08083DF91CF911F91AF
:104900000F91089581E08083B9CF80910503909144
:104910000603B8CF0F931F93CF93DF938C01EB0166
:1049200063E073E08C2F0E940316892B71F4DD275E
:10493000C15DDD4F8881F801128218828330E9F071
:1049400048F4813059F0823081F0DF91CF911F918E
:104950000F9108958430B1F08530B9F78091030349
:1049600090910403009789F306C08091050390910C
:104970000603009799F3FCDEE8CF8091070390913E
:104980000803F7CF8091090390910A03009799F7E4
:104990002091030330910403809105039091060355
:1049A00021153105F9F2009731F7C901E4CFCDB7F0
:1049B000DEB7AC970FB6F894DEBF0FBECDBF85B79C
:1049C000806885BF85B7806885BF84B7877F84BFCF
:1049D0000FB6F894A895809160008861809360007C
:1049E000109260000FBE80E890E00FB6F8948093BC
:1049F0006100909361000FBE81E08093480180EBDD
:104A000095E09093DD018093DC010E94D8050E941F
:104A100084150E94CC090E94420A8091E2008460C1
:104A20008093E200789480917302811599F08091CF
:104A3000E9001091EC008F70179511271795182B2E
:104A40001092E9008091E80083FD0E94110D1F7013
:104A50001093E90082E084BD93E095BD9AEF97BD85
:104A600080936E001092AB021092AC021092AD02D5
:104A70001092AE020E94F714811102C00E94D21659
:104A800088EC90E02091E30027FD0EC0AFE3BCE985
:104A90001197F1F700C000000197A1F70E94CC091F
:104AA0001092730280E001C081E08093A90280939C
:104AB000AA02809300018111FCD7809100018091AE
:104AC000000190E0811101C096E09093440286E0DD
:104AD000891B8093430202E611E0F80181918F0166
:104AE0008F3F11F00E94B205F1E008361F07A9F7C9
:104AF00008E611E05EE6E52E51E0F52ED8018D9135
:104B00008D018F3F11F00E94B205E016F106B1F75A
:104B10008CE0E5E6F2E0DF01282F1D922A95E9F707
:104B2000E7E3F2E0DF011D928A95E9F780E090E08B
:104B30000E94552F833E9E4F21F40E94F71481114D
:104B400029C063EE7EEF80E090E00E94832F60E05A
:104B500082E090E00E94692F81E08093200461E070
:104B600083E090E00E94692F60E074E184E090E0CF
:104B70000E94832F0E94D21640E050E0BA018FE0DD
:104B800090E00E947B2F40E050E0BA0183E190E08A
:104B90000E947B2F82E090E00E944D2F809347027D
:104BA00084E090E00E94552F90936A0480936904FA
:104BB0000E947010EFEFF6E721E0E150F040204056
:104BC000E1F700C000000E9470108091650280FF34
:104BD00008C06FEF7FEF80E090E00E94832F0E947B
:104BE000120983E090E00E944D2F0E94DC02809128
:104BF000A902811101C060D781E091E09093D602B3
:104C00008093D50280917302853049F480917302BC
:104C1000853009F450C00E94D00C0E9490060E947A
:104C2000701008E412E045E6E42E42E0F42ED701CD
:104C3000F80191918D9124E532E02E173F0709F498
:104C40006EC09817B1F38090A902D12CD701CD90F6
:104C50007D01F80191908F019C1431F19C24B12CBD
:104C6000AA24A394892D8A218115B9F08114A9F071
:104C7000B982DA820E9456079C838B83F1E0FD8320
:104C800091E08C2D8A21811101C090E09E834981A1
:104C90005A816B817C818D8179DCB394AA0C26E0EA
:104CA000B212E0CFF801C292D3943CE0D312CECF3F
:104CB0000E94B90837C080917302843021F11092AC
:104CC000450288E190E0A0E40FB6F894A89580939F
:104CD00060000FBEA093600083B7817F846083BFB4
:104CE00083B7816083BF7894889583B78E7F83BFB5
:104CF0000FB6F894A8958091600088618093600059
:104D0000109260000FBE0E947010E5E6F2E0819103
:104D10008111E1C4B2E0E137FB07C9F777CF9813FF
:104D200092CFE3DC8091A902811509F478C000914B
:104D30008E0310918F030115110591F1C090580257
:104D4000D0905902E0905A02F0905B020E94AD08A8
:104D50006C197D098E099F09C0905402D0905502AC
:104D6000E0905602F09057026C157D058E059F0568
:104D7000B8F0C8010E94610C10928E0310928F034C
:104D8000109258021092590210925A0210925B022D
:104D9000109254021092550210925602109257022D
:104DA000E0901604F0901704E114F10439F1C0907A
:104DB0001804D09019040E9456078C010C191D0983
:104DC000C7010E94181680179107C0F4209116049D
:104DD00030911704C9019927287F3327232B09F025
:104DE0002FC134E0880F991F3A95E1F78A569C4FFE
:104DF000DC0115962C9122FF0E94F00F80910D038B
:104E0000811569F00E94560720910E0330910F031F
:104E1000821B930B8F3F9F4710F40E94C70C86E0C4
:104E2000EDEFF2E0DE01119601900D928A95E1F727
:104E3000B090FE02D090FF02F0900003C0900103FA
:104E4000E09002031092FF021092000310920103FF
:104E5000109202038F2D8D29811509F441C0009114
:104E60005E0210915F020E9456079C01201B310BCD
:104E70009091FB02911509F429C42531310580F187
:104E80009F3F19F09F5F9093FB02D11459F00E944D
:104E9000460691E01D140CF09FEF899F802D112490
:104EA0008093FF02F11459F00E94460691E01F140E
:104EB0000CF09FEF899F802D112480930003809137
:104EC000FF02811569F010910003111549F00E944D
:104ED00038068093FF02812F0E94380680930003DA
:104EE0008C2D8E29811509F441C000915C0210912E
:104EF0005D020E9456079C01201B310B9091FA0223
:104F0000911509F4DEC32135310580F19F3F19F079
:104F10009F5F9093FA02C11459F00E94660691E0D7
:104F20001C140CF09FEF899F802D112480930103A6
:104F3000E11459F00E94660691E01E140CF09FEFF8
:104F4000899F802D11248093020380910103811594
:104F500069F010910203111549F00E943806809300
:104F60000103812F0E943806809302038091FE0284
:104F70008B1119C08091FF02811511F08D1113C0A2
:104F800020910003211511F02F110DC09091020303
:104F9000911511F09E1107C030910103311103C02A
:104FA000822B892B81110E94C90786E0FE01319670
:104FB000ADEFB2E001900D928A95E1F70E94900664
:104FC00090916002891721F0809360020E94AD08E1
:104FD00080917302843009F015CE83E08093E9005C
:104FE0008091E80082FF0ECE8091E80090E085FF7E
:104FF00005C00E949B09811531F191E08091E80084
:105000008B778093E800911509F4FCCD0091B102F3
:105010001091B202E9810115110589F1EE3F09F005
:1050200050C08A81833020F08550833008F049C019
:10503000EA81EE3008F045C0F0E0EE50F04DD6C603
:1050400080E090E0D5CE00E210E0FE0131967F01D5
:105050008091E80085FD0AC08091E8008B778093FD
:10506000E8000E949B09811599F3C7CF8091F10058
:10507000D7018D937D010150104051F7BECFE4312F
:1050800048F4E11549F0E150E33130F4F0E0E0504C
:10509000F04DACC6EE3F61F28FEF898312C01A82E9
:1050A00089E08B830EC08A81823081F08330B1F039
:1050B000813091F70E94AD089FD66B837C838D83EE
:1050C0009E83CE0101960E94EB099CCD88E290E080
:1050D000E4D61B821C821D828E83F3CF80917102E5
:1050E00090917202892B69F38CE0E5E6F2E0DE0133
:1050F000139601900D928A95E1F7E3CF8A81823071
:1051000059F66B817C818D819E8176D688E290E014
:10511000E0D6D7CF4C816B818A810E941D149827DD
:10512000892798279E838D83CCCF2D813E8132277E
:10513000232732274C816B818A810E94720BC1CF59
:105140000E941015BECF80E18A83BBCF1A8287EF01
:10515000A8CF8C818D3108F0B4CF8A809B809824B1
:1051600089249824A12CB12C8E010F5F1F4F780148
:10517000E80EF11C0E151F0509F4A3CF80E0B7EF70
:105180008B169104A104B10420F4C401875F9C4FE5
:1051900084D6F80184830F5F1F4FFFEF8F1A9F0A99
:1051A000AF0ABF0AE7CF8091710290917202892BFA
:1051B00009F487CF8C818D3108F083CF882E912C14
:1051C000A12CB12CCA80DB80DC24CD24DC24E12C92
:1051D000F12C8E010F5F1F4F412C512C32014814CE
:1051E00059046A047B0408F06CCF27EFC216D1047F
:1051F000E104F10438F4D80114966C91C601875F7C
:105200009C4F67D6BFEF4B1A5B0A6B0A7B0AEFEF26
:10521000CE1ADE0AEE0AFE0A0F5F1F4FE0CF0E9491
:1052200098164FCF84E090CF8C818D3108F049CF14
:10523000882E912CA12CB12CCA80DB80DC24CD24BB
:10524000DC24E12CF12C412C512C32018E010B5F1E
:105250001F4F481459046A047B0408F032CF80E0E1
:10526000F0E4CF16F2E0DF06E104F10418F4C60121
:10527000899613D6D8018D938D01BFEF4B1A5B0A27
:105280006B0A7B0AEFEFCE1ADE0AEE0AFE0AE1CFC6
:105290002C81022F10E02D3108F013CF8A819B81E1
:1052A0009827892798272C01612C712C8034F2E0F3
:1052B0009F0708F006CF822E912CA12CB12C40E440
:1052C00052E060E070E04419550966097709421719
:1052D00051056105710508F4F4CE209171023091F9
:1052E0007202232B09F03EC01C0129E2220E311C60
:1052F00080FBEE24FF24E0F880FF0BC08896CDD51C
:105300009D8189279827892781159C4711F48FEF64
:105310008D83D501C401840D951DA61DB71D80FF89
:1053200019C0680181E0C81AD108DE011596AC0DDC
:10533000BD1DBCA7ABA7C101800F911FAED5EBA5CA
:10534000FCA5908181159C4721F48FEFABA5BCA5EE
:105350008C938601FE013196EE0DFF1D2FEFE016B6
:10536000F10638F08E010F5F1F4FC12CD12C760152
:1053700025C09481858181159C4711F42483258360
:1053800032E0E30EF11C3296EACF80E4481682E068
:1053900058066104710430F4D80114966C91C2016E
:1053A000899697D5BFEFCB1ADB0AEB0AFB0AEFEF22
:1053B0004E1A5E0A6E0A7E0A0F5F1F4FC814D90488
:1053C000EA04FB0410F37DCE809171029091720289
:1053D000892B09F476CECE0101960E94EB09FFEFEE
:1053E00021EE34E0F15020403040E1F700C00000F1
:1053F000F6CB88E0EAE4F1E0DE01919601900D92AF
:105400008A95E1F7FE0132968FE1DF011D928A95C0
:10541000E9F786E0898388E07F96DE01159669CEFC
:105420008CE2898381E08A831B821C824ACE8B8135
:105430009C81092E000CAA0BBB0B25E0880F991F3D
:10544000AA1FBB1F2A95D1F7AC01BD01405E5F4F7B
:105450006F4F7F4F481759076A077B0708F431CE13
:105460008C32E1E09E07A105B10508F02ACE4D324D
:10547000F1E05F076105710520F04CE251E060E06A
:1054800070E0481B590BBC016D537C4FCE01019657
:10549000CED417CE4AE150E06FEF70E0CE01079610
:1054A000E5D48091710289830A831B821C8281E08A
:1054B0008D8312CE81E090E09093B2028093B1028E
:1054C00082E390E090936402809363020E94560707
:1054D0009093620280936102F4CD0115110581F170
:1054E000D0906502C0906602E0906102F090620286
:1054F0000E9456078E199F098536910540F1C1FE1D
:1055000026C0D0FE24C00E9456079093620280936A
:10551000610280916302909164020197909364020A
:1055200080936302892B61F41092B2021092B1024F
:1055300081E090E0909372028093710200E010E0AD
:105540008091710289830A8380916302AACD82E3EC
:1055500090E09093640280936302F2CF1092720203
:1055600010927102AECD40E250E06FEF70E0CE01DC
:1055700001967CD4A6CD8B81823009F450C078F49A
:10558000811136C0FE0132968EE1DF011D928A95AF
:10559000E9F788E089838B8383E088A392CD853007
:1055A00009F472C0863009F08CCD1C818AE0FE01BE
:1055B0003596DE01919601900D928A95E1F78BA1C7
:1055C0009CA10E94CB059CA38BA38FEF183060F4A5
:1055D000FAE01F9FB001112467547D4F4AE050E06C
:1055E000CE01819694D480E089830E94841569CD90
:1055F0008C819AE0F92E8E010F5D1F4FF8012F2D3F
:1056000011922A95E9F7B8010E9403168983F801DF
:10561000DE01129601900D92FA94E1F752CD1C81B1
:105620008AE0FE013596DE01919601900D928A95F1
:10563000E1F789A19AA10E94CB059AA389A38BA126
:105640009CA10E94CB059CA38BA38DA19EA10E942F
:10565000CB059EA38DA38FA198A50E94CB0598A7EB
:105660008FA38FEF183060F43AE0139FB00111243C
:1056700067597D4F4AE050E0CE01819648D480E0E2
:1056800089830E94D8051DCD2C816AE0CE018196C8
:10569000DC01E62F1D92EA95E9F7283080F4629F3D
:1056A000B001112467547D4F4AE050E0E6D380E01A
:1056B00089838AE0FE01B196DE0112961ACD8FEF42
:1056C000F7CF2B30310508F023CC50CC2B303105EF
:1056D00008F0D8CB05CC80914602811509F496CA12
:1056E000E0E1E9BDF2E1F9BD09B400FEFDCF809132
:1056F000D8008F7D8093D8008091E00082608093F5
:10570000E0008091E00081FDFCCF0E94D00C7ECAB9
:105710001F921FB61F9211248F939F93AF93BF9335
:1057200080914502811113C0809126029091270239
:10573000A0912802B09129024196A11DB11D80932C
:10574000260290932702A0932802B0932902BF91CA
:10575000AF919F918F911F901FBE1F9018957894C5
:105760001F921FB61F9211248F939F93AF93BF93E5
:105770008091260290912702A0912802B0912902DF
:105780000196A11DB11D8093260290932702A0933C
:105790002802B0932902BF91AF919F918F911F90E2
:1057A0001FBE1F9018951F920F920FB60F921124D3
:1057B0002F933F934F935F936F937F938F939F9319
:1057C000AF93BF93EF93FF938091E10082FF09C0F5
:1057D0008091E20082FF05C08091E1008B7F809381
:1057E000E1008091DA0080FF24C08091D80080FF22
:1057F00020C08091DA008E7F8093DA008091D900FA
:1058000080FFA9C080E189BD82E189BD09B400FEA5
:10581000FDCF81E08093730280911502811109C050
:105820000E94CC090E94420A8091E2008460809329
:10583000E2008091E10080FF1AC08091E20080FFC9
:1058400016C08091E2008E7F8093E2008091E2009A
:1058500080618093E2008091D80080628093D800BC
:1058600019BC85E08093730283E0809348018091A6
:10587000E10084FF2FC08091E20084FF2BC080E113
:1058800089BD82E189BD09B400FEFDCF8091D800B9
:105890008F7D8093D8008091E1008F7E8093E1001E
:1058A0008091E2008F7E8093E2008091E20081602F
:1058B0008093E20080911402811509F452C084E0C3
:1058C0008093730280917302843009F052C082E0A9
:1058D000809348018091E10083FF2CC08091E20019
:1058E00083FF28C08091E100877F8093E10082E000
:1058F00080937302109214028091E1008E7F809356
:10590000E1008091E2008E7F8093E2008091E200CE
:1059100080618093E20042E060E080E00E94120A31
:105920008091F00088608093F00081E080934801CE
:1059300080934701FF91EF91BF91AF919F918F911C
:105940007F916F915F914F913F912F910F900FBE7B
:105950000F901F90189519BC1092730210921502A7
:1059600068CF8091E30087FF02C083E0A9CF81E088
:10597000A7CF81E0ADCF1F920F920FB60F921124E7
:10598000EF92FF920F931F932F933F934F935F9349
:105990006F937F938F939F93AF93BF93CF93EF9327
:1059A000FF9309EE10E0F8018081C091EC008F7048
:1059B000C795CC27C795C82B108280EFE82EF12C15
:1059C000F7018081877F808378940E94110DF80110
:1059D0001082F701808188608083CF70F801C083D6
:1059E000FF91EF91CF91BF91AF919F918F917F9157
:1059F0006F915F914F913F912F911F910F91FF9068
:105A0000EF900F900FBE0F901F9018958EE1489B5E
:105A100002C08A95E1F7489BFECF0895589880E22E
:105A20008A95F1F7589A0895FC012BE02A95F1F731
:105A300028E090E080E031E040E14A95F1F7880FFE
:105A4000489B02C08160932742E04A95F1F700002D
:105A500040E14A95F1F72A9579F720E12A95F1F787
:105A600029B132E03A95F1F7000040E14A95F1F7AB
:105A7000217092272081920F90830895A1E0B0E0D9
:105A8000E3E4FDE275C119828C017C01E60EF11C94
:105A9000BDDFCE010196C8DFF80181938F01EE15BD
:105AA000FF05B1F781E09981911180E02196E6E050
:105AB0007BC1509A589A08955098589AE89AE9E606
:105AC000F0E080818C7F808308956150770B91E0B6
:105AD00001C0990F6A95EAF7692F90E021E0611102
:105AE00008C0911599F0589A80E28A95F1F7589874
:105AF0000895362F3823311539F0589A922730E21D
:105B00003A95F1F76695EBCF5898F9CF5898ECCFC6
:105B1000FF920F931F93CF93DF93EC018C01060F3D
:105B2000111DF9907BDF68E08F2DCFDFC017D10703
:105B3000C1F7CDB7DEB7E5E038C11F920F920FB6BF
:105B40000F9211240F931F932F933F934F935F93C3
:105B50006F937F938F939F93AF93BF93EF93FF9335
:105B6000CF93DF930F92CDB7DEB719824FDFCE010F
:105B700001965ADF082F069506950695982F92955F
:105B80009570202F2570920F292F2370969596954A
:105B9000920F982797708981892B811509F058C039
:105BA000083008F055C080E18A95F1F7589A509A6C
:105BB00082E08A95F1F700C0589888E0089F80013C
:105BC0001124D801A35FBE4F1696ED91FC91179753
:105BD0003097A9F060916E0170916F0114962D912C
:105BE0003C911597260F371F11968D919C91129716
:105BF000680F791F13964C9113978C910995F801B2
:105C0000E35FFE4F6381611549F020916E01309191
:105C10006F0184819581820F931F7ADFFFDE80E11F
:105C20008A95F1F758985098589A80E18A95F1F73B
:105C3000F801E35FFE4F6081611549F020916E012C
:105C400030916F0181819281820F931F17DFDEDE19
:105C50000F90DF91CF91FF91EF91BF91AF919F9105
:105C60008F917F916F915F914F913F912F911F91F4
:105C70000F910F900FBE0F901F9018950F931F93C9
:105C8000CF93DF938C0108970CF05EC0F894509A84
:105C9000589885E08A95F1F70000C02FC695C57029
:105CA000802F8570C80F8C2F8370C695C69593E0A2
:105CB000000F111F9A95E1F7C80FC8018C2BEC015A
:105CC000ADDE00C068E08C2F00DF90E19A95F1F71F
:105CD0005098589A489B31C087E090E048992FC06F
:105CE000F801E35FFE4F6381611559F020916E0169
:105CF00030916F0184819581820F931FBFDE8115E2
:105D000001F184DE80E28A95F1F75898509A90E18B
:105D10009A95F1F7F801E35FFE4F6081611549F054
:105D200020916E0130916F0181819281820F931FCA
:105D3000EFDE74DE789481E008C000C0CBCF01971D
:105D400049F4509A589A789480E0DF91CF911F914E
:105D50000F91089500C0C2CF2F923F924F925F9251
:105D60006F927F928F929F92AF92BF92CF92DF926B
:105D7000EF92FF920F931F93CF93DF93CDB7DEB7D0
:105D8000CA1BDB0B0FB6F894DEBF0FBECDBF099464
:105D90002A88398848885F846E847D848C849B84BB
:105DA000AA84B984C884DF80EE80FD800C811B81C9
:105DB000AA81B981CE0FD11D0FB6F894DEBF0FBEF8
:105DC000CDBFED01089597FB072E16F4009406D081
:105DD00077FD08D018D007FC05D03EF4909581954A
:105DE0009F4F0895709561957F4F0895EE0FFF1FA7
:105DF0000590F491E02D0994692796276927782763
:105E0000872778270895AA1BBB1B51E107C0AA1F4B
:105E1000BB1FA617B70710F0A61BB70B881F991F4B
:105E20005A95A9F780959095BC01CD010895FB0185
:105E3000DC0102C005900D9241505040D8F7089502
:105E4000FB01DC0104C08D910190801921F44150C7
:105E50005040C8F7881B990B0895FB01DC0102C074
:105E600001900D9241505040D8F70895DC0101C0D7
:105E70006D9341505040E0F70895DC01CB01FC01E7
:105E8000F999FECF06C0F2BDE1BDF89A319600B493
:105E90000D9241505040B8F70895F999FECF92BD48
:105EA00081BDF89A992780B50895A8E1B0E042E055
:105EB00050E0E5CFDC01A40FB51F4150504040F049
:105EC000CB01840F951F2E9105D041505040D8F73B
:105ED0000895262FF999FECF92BD81BDF89A0197BA
:105EE00000B4021639F01FBA20BD0FB6F894FA9A22
:105EF000F99A0FBE08950396272FECDFEADF252FCE
:105F0000E9DF242FE7CF0196272FE4DFE2CFDC0182
:105F1000CB0102C02D9105D041505040D8F70895D3
:105F2000262FF999FECF1FBA92BD81BD20BD0FB6B5
:105F3000F894FA9AF99A0FBE01960895F894FFCF53
:105F4000FE07030805080A081A081A081A081A089A
:105F50001A081A081A081A080C0810081308180852
:105F600028082E083208EE0D140E1A0E140E1A0E02
:105F70006C0E8D0E1A0E930FA00FF51C5D1DFD1CEF
:105F8000C71CCB1C011DCF1C051D111DDB1C561D84
:105F9000DF1C151DE31C191D3E1DE71C1D1D451DA5
:105FA000ED1C231D2B1DD31C091DD71C0D1DF11C21
:105FB000271D351D4E1D541DC11CF91C641D931C4D
:105FC000991C861C8D1C9F1CA51CAB1CBF1EBF1ED4
:105FD000F61EF61EA61FC11F1A1F1A1FC61F392044
:105FE0004A204A20F929102A172A612861284A2ABA
:105FF0005A2A6D2AAE2AB32A612861286128BB2A51
:106000004F2853287E288A289528A0284C284C28D9
:106010004C284C28E429A328A628A928D3280F29EE
:0660200012291429482991
:10602600015307FD0A130B180B1D0BF40A000000A1
:106036000100000000000000060100000006070045
:106046000000000000040D00000000000001110027
:106056000000000000011200000000000004130010
:106066000000000000000001000109B2188732BBE1
:10607600665F004422B684016201AC008A02A30274
:10608600C3029135333236F6C6976694F4F592021A
:10609600E200E900EA00B500B600B700CD008301D2
:1060A600CC008A01920194012102230224022502D6
:1060B600260227022A02B300B4006F0070009F0177
:1060C600CB019F02A002E200E900EA00B500B6009B
:1060D600B700CD008301CC008A0192019401210210
:1060E600230224022502260227022A02B300B40054
:0C60F6006F0070009F01CB019F02A00210
:00000001FF
